:030000000211FBEF
:03000B000200C12F
:03002B000203EBE2
:03005B0002053D5E
:0300730002053350
:1000800002030406080C10182030406080020304AC
:1000900006080C101820304080FF0406080C1018C9
:1000A0002030406080A0C000000001010003020277
:1000B000010D0D040506020D0505050D06040502DA
:1000C00002C2AFC0D0C0E0205A0D302F02E473301E
:1000D000600280F90203D7306306C2B1C287C281D1
:1000E00085258AC25AE525F4700221CA056130606F
:1000F00013206A19758B00D0E0D0D0C2B1C287C27C
:1001000081D2AF32C2B1C287C2810201BAD26EC2FD
:100110006FE565601CC3E5611495654014C26ED23D
:100120006FC3E561956450030201BA756100020175
:10013000BA206C14C2B1C287C2817406D5E0FDD268
:1001400082D286D2800201BAD26FC2B1C287C28186
:10015000E53D20E23420E1127406D5E0FD20750271
:10016000D280307502D2820201BA20E0127406D524
:10017000E0FD207502D280307502D2820201BA748D
:1001800006D5E0FDD2860201BA20E11F20E00A7404
:1001900006D5E0FDD2860201BA7406D5E0FD2075D1
:1001A00002D282307502D2800201BA7406D5E0FD17
:1001B000207502D282307502D280758B00D0E0D0DB
:1001C000D0C2B1C287C281D2AF32D0E0D0D0D2AFDC
:1001D0003261D7E525600A207502D2B1307502D2AE
:1001E00081C28761D7E5256002D287207502C2816E
:1001F000307502C2B161D7E525600A207502D2814F
:10020000307502D2B1207502C2B1307502C281616F
:10021000D7207502C282307502C280E525600A20AF
:100220007502D2B1307502D281207502C28030755C
:1002300002C282C28761D7207502C282307502C2B3
:1002400080207502C280307502C2827406D5E0FD3E
:10025000E525600A207502D2B1307502D281C287CD
:1002600061D7207502C282307502C280E525600A1E
:10027000207502D2B1307502D281C286C28761D7A1
:10028000207502C282307502C280C2867406D5E033
:10029000FDE525600A207502D2B1307502D281C217
:1002A0008761D7C286E5256002D287207502C282A7
:1002B000307502C280207502C281307502C2B16100
:1002C000D7C286207502C282307502C2807406D5FC
:1002D000E0FDE5256002D287207502C281307502FB
:1002E000C2B161D7C286E5256002D287207502C2FD
:1002F00080307502C282207502C281307502C2B19F
:1003000061D7C286207502C280307502C28274062F
:10031000D5E0FDE5256002D287207502C2813075E7
:1003200002C2B161D7207502C280307502C282E577
:1003300025600A207502D281307502D2B1C28620B2
:100340007502C2B1307502C28161D7207502C280C8
:10035000307502C282C2867406D5E0FDE525600ACA
:10036000207502D281307502D2B1207502C2B1303F
:100370007502C28161D7207502C280307502C282C7
:10038000E525600A207502D281307502D2B1207550
:1003900002C282307502C280207502C2B13075027D
:1003A000C28161D7207502C280307502C282207579
:1003B00002C282307502C2807406D5E0FDE5256078
:1003C0000A207502D281307502D2B1207502C2B105
:1003D000307502C28161D7E525F4F58A758B007509
:1003E0006000D25AD0E0D0D0D2AF32C2AFC0D0C0BD
:1003F000E0D2D3C2CEE528600A741F552E6049159D
:1004000028814878007900E580307601F430E502F3
:1004100078FF53DACF20760343DA2030760343DACD
:1004200010C2D8C269E580307601F430E50279FF68
:10043000C3E89970CE305903752818741F552E6083
:10044000037528188858D268E52960041529815B4E
:10045000741F552E600543DA01C2D820680281ED71
:10046000E558F8C268741F552E60367982B704319A
:0F047000C3E894F0400374F0F8E8C4540F28F880
:10047F007984B7030281A1C313C313872120080214
:10048F00C313200A06C3C898F881A128F850037433
:10049F00FFF8C3E8955F5003E55FF8E52C5406704D
:1004AF003D882230630AC3E522955C4003855C22B8
:1004BF007882B60429C3E5229524401278A096408D
:1004CF000DE52426F52450097524FF0204E085224A
:1004DF0024852425C3E524955C4003855C2520CF26
:1004EF0009D0E0D0D0C2D3D2AF32C2CF7801E52845
:1004FF006008741F552E70021528C3E558940140EB
:10050F0005755B00A11CE55B046002055BE55DC33F
:10051F00240A5005755DFFA12AF55DD0E0D0D0C249
:10052F00D3D2AF32C2AF53917FC258D2AF32C2AF24
:10053F00C0D0C0E0C0F0D2D3A8FBA9FCC2D83069AC
:10054F0002A1A053DACF20760343DA1030760343AB
:10055F00DA20D269E580307601F420E502A17488B3
:10056F00268927E14053DACF20760343DA2030760D
:10057F000343DA10C2D8C269741F552E7002E126E8
:10058F007800E580307601F430E502E1268858E105
:10059F002653DACF20760343DA2030760343DA107E
:1005AF00C269205902C15A53DACF20760343DA10B9
:1005BF0030760343DA20C2D8D26988538954C3E80E
:1005CF009551F8E99552F9E4FB7AFAC3E894C8E932
:1005DF0094005008E4D2E4FB7A0AC12DC3E8946872
:1005EF00E994015008E4D2E3FB7A0FC12DC3E894DC
:1005FF00D0E994025008E4D2E2FB7A1EC12DC3E881
:10060F0094A0E994055008E4D2E1FB7A3CC12DC3D4
:10061F00E89498E994085006E4D2E0FB7A78C3E8AE
:10062F009555FCE99556FD30E708ECF42401FCEDF7
:10063F00F4FD7557007008C3EC9A50037557018885
:10064F00558956A853A95488518952C3E89526F85D
:10065F00E99527F9307402C1F9307302C1F930728C
:10066F0002C1F2E9C313F9E813F8307102C1F2E9DC
:10067F00C313F9E813F8307002C1F2E9C313FDE8B0
:10068F0013FC205918C3EC941CED9402400302078D
:10069F0026ED7009C3EC94C8500302074074002084
:1006AF0077037896E624FAFEE43400FFC3EC9EFC51
:1006BF00ED9FFD500678007900C1F9C3EC94FFED72
:1006CF009400400678FF7900C1F9EC856CF0A4C561
:1006DF00F0A2F733F87900400302071578FF79008D
:1006EF00020715E9C313F9E813F830740EE9600235
:1006FF0078FFC3E81338F8E43400F9C3E894FFE94E
:10070F009400400278FF8858D268205902E126747D
:10071F001FF4552E4BF52E752818741F552E700388
:10072F0075280A305902E140741F552E600353DAC1
:10073F00FE752906741F552E700375290AD0F0D047
:10074F00E0D0D0C2D3D2AF327901E16F7903E16F3C
:10075F00790AE16F791EE16F7964E16F79C8E16F12
:10076F007817E4D5E0FDD8FAD9F6227A147B78020F
:10077F0007967A107B8C0207967A0D7BB402079648
:10078F007A0B7BC8020796AC257525017902B275E5
:10079F00E4C286D5E0FDE5256002D287D5E0FDC233
:1007AF0087D5E0FDD286D5E0FDE525600A207502EC
:1007BF00D2B1307502D281E56DD5E0FD207502C250
:1007CF00B1307502C2817496D5E0FDD9C1EAF8D572
:1007DF00E0FDD8FBDBB1C2868C2522C37C007D00F7
:1007EF0075F00005F0EA33FAEB33FB50F6EB13FB31
:1007FF00EA13FAC3E9FFE8FEE89AF8E99BF9500417
:10080F00EFF9EEF8B3EC33FCED33FDD5F0DFEDF996
:10081F00ECF822E889F08A20D2D4F8A9F07B0030D6
:10082F00F70B7BFFF42401F8E9F43400F9E8852095
:10083F00F0A4ADF0F8E98520F0A4AFF0FEED2EF9AD
:10084F0074003FFA7C04C3EA13FAE913F9E813F8CA
:10085F00DCF48BF030F70AE8F42401F8E9F4340003
:0F086F00F9E889F0C2D4F8A9F0227882B6040320
:10087E000208D6C3E5589401400302089E8522243F
:10088E00E4F53FF540F541F542F543F5480208D64B
:10089E007882E6FC754801E522F523783879C7AAF7
:1008AE003BAB3CC3EB13FBEA13FAEC146013C3EB44
:1008BE0013FBEA13FAEC14146007C3EB13FBEA13F1
:1008CE00FA1207EA883F894022E5486034C3E53FC3
:1008DE009523F8E5409400F9500CC3E89480E99410
:1008EE00FF401602090BC3E8947FE99400500302FF
:1008FE00090B787F790002090B788079FF8844898B
:10090E004522E5486058E5442541F8E5453542F96C
:10091E00854520E4300701F43543FA30E709C3EA90
:10092E0094F0401502094DC3EA940F500302094D8D
:10093E0078FF79FF7A0F02094D780079007AF0C3BB
:10094E00E524955C5006E52460092166E54520E71F
:10095E000D2166E54530E706884189428A4322E546
:10096E004870030209D0789EE6FAC3E54433F8E5F1
:10097E004533F91122E930E70BC3E89480E994FF7F
:10098E00401321A7C3E8947FE99400500221A77871
:10099E007F790021A7788079FFE820E715C3E5234A
:1009AE0098F84009C3E8940140030209CE78010289
:1009BE0009CEE8F424012523F840030209CE78FF7E
:1009CE00884622E5487003020A32789FE6FAA8426A
:1009DE00A9431122E930E70CC3E89401E994FF40E2
:1009EE0016020A09C3E894FFE994005003020A09AB
:1009FE0078FF7900020A09780179FFE920E715C32B
:100A0E00E54698F84009C3E894014003020A30789D
:100A1E0000020A30E8F424012546F84003020A30A9
:100A2E0078FF8824227883E6F520120F6F75E89000
:100A3E00E5E820ECF0A8BDA9BE1210047568557546
:100A4E006900C3740013FD745513FC74552CFC74AB
:100A5E00003DFDECFAEDFBC3E89AE99B4014E56816
:100A6E002455F568E5693400F569EA2CFAEB3DFB8F
:100A7E0080E5AE68AF69C3E56913F9E56813F8C39D
:100A8E00E913F9E813F8E56828F566E56939F567BD
:100A9E007A03C3E913F9E813F8DAF7AA201A7009F2
:100AAE00756800756900020AC71AEA6008EE28FE2A
:100ABE00EF39FFDAF88E688F692275E89022788315
:100ACE00E6FFE5E820ECF7A8BDA9BE056AC3E56A16
:100ADE0094084052756A00E97007E56B601B020AC4
:100AEE00FBC3E8956B6010E56B5006600C14020BAF
:100AFE00070460F9020B07E56BF56BC394A8F84089
:100B0E0021755CC0C3E89405F84017755C80C3E896
:100B1E009405F8400D755C40C3E89405F8400375E4
:100B2E005C0075BB0622EFC39401601BC3E894FF03
:100B3E00E994035012C3E89568E995695009E55C9C
:100B4E00600C155C020B5CE55CF46002055CA85C55
:100B5E00C3E524985002A8248825C3E525955D4059
:100B6E000B855D25E55DF46003855D5CC3E56AB4C8
:100B7E00070375BB1E22306102783230620278782C
:100B8E00E52C5406601FE879A187F0A4C5F0A2F702
:100B9E0033F8C3E8955C4002A85C88228824882537
:100BAE00306102885E22788FE6FFC3EF94055018FD
:100BBE00C3EF94045020C3EF94035028C3EF940264
:100BCE005030C3EF940150387533A075340F75351E
:100BDE003C753605811C7533C075341275354075FC
:100BEE003606811C7533707534177535D07536071A
:100BFE00811C75334C75341D7535C4753609811CD1
:100C0E007533287534237535B875360B811C8533CD
:100C1E004F853450753B00753C0822A84FA95002F1
:100C2E000C34A849A94A759100C3E498F594E49947
:100C3E00F595759104D25875C820A8CCA9CD75C864
:100C4E0024AA39AB3A8839893AC3E89AF8E99BF96C
:100C5E00AA3BAB3CC3EB13FDEA13FCC3ED13FDEC57
:0F0C6E0013FCC3EA9CFAEB9DFBEA28FAEB39FB77
:100C7D008A3B8B3C400122753BFF753CFF2230586F
:100C8D0002818B759100C3E4954BF594E4954CF579
:100C9D0095759104D258227892E6FF7E10305B0252
:100CAD007F053063047F037E00A93CA83B7A04C313
:100CBD00E913F9E813F8DAF7C3E89EF8E99400F9B7
:100CCD004009C3E89402E9940050047802E4F9E97C
:100CDD00FBE8FAC3E913FDE813FCC3EF9403602EA0
:100CED00EF20E00DE82CF8E93DF9ECFAEDFB020DF3
:100CFD0008E828F8E939F97A02E4FBC3EF940340D8
:100D0D000D8A4D8B4E8849894A8C4B8D4C22884DCE
:100D1D00894E8A498B4A8C4B8D4C22305802A12822
:100D2D00759100C3E4953BF594E4953CF59575916B
:100D3D0004D25822753E00752000020D50753E00FC
:100D4D00752040D2AF053E20580122759D00E53C2F
:100D5D00C313C313F8086030306A06C313C313F806
:100D6D0008C3E8940A4002780A306D08C3E8940479
:100D7D0040027804C3E53C9408400D759D02C3E51F
:100D8D003C94104003759D03205803D2AF22791E69
:100D9D00206D02790AD2AF0000C2AF205A0A793C09
:100DAD00206D027914306FE03063027978C3E58BE2
:100DBD009920630240F740D0E59BF45440B52002E2
:100DCD00A150D8C4D2AF22C25B789CE6146007E56F
:100DDD003E147002D25B30630B0538205810753805
:100DED0000020DFB2058071581158102175622753B
:100DFD009100C3E4954DF594E4954EF595759104E8
:100E0D00D25822AE25305B4F78A3E6FFBF010BD23F
:100E1D005C752500C2B1C287C2819190305C0375AB
:100E2D002500305802C129BF020BD25C752500C2C6
:100E3D00B1C287C28178A2B6010D9190305C037565
:100E4D002500305802C149BF030BD25C752500C285
:100E5D00B1C287C281B1FC305C03752500305802E8
:100E6D00C164305B04C25C8E2522C2AFC286206A8B
:100E7D0003020E9690034B306E0F207502C2803028
:100E8D007502C2827406D5E0FD207502D2823075DE
:100E9D0002D280759F02753D02D2AF22C2AF206A89
:100EAD0003020ECB900302306E17C286207502C26C
:100EBD0080307502C2827406D5E0FD020ECE90011F
:100ECD00E5207502C281307502C2B1305A06E525A2
:100EDD006002D287207503759F03307503759F01DE
:100EED00753D03D2AF22C2AF207502C282307502AA
:100EFD00C280206A03020F129002C1306E07C286B3
:100F0D007406D5E0FD207502D280307502D28220A4
:100F1D007503759F01307503759F03753D04D2AF41
:100F2D0022C2AF206A03020F50900280306E17204C
:100F3D007502C282307502C280C2867406D5E0FD8C
:100F4D00020F539001D3C287305A0EE525600A2057
:100F5D007502D2B1307502D281759F02753D05D2F1
:100F6D00AF22C2AF207502C280307502C282206AE4
:100F7D0003020F96900237306E0F207502C2823039
:100F8D007502C2807406D5E0FDD286207503759F6B
:100F9D0003307503759F01753D06D2AF22C2AF2098
:100FAD006A03020FD49003A4306E1F207502C28213
:100FBD00307502C280207502C280307502C2827403
:100FCD0006D5E0FD020FD79001F7207502C2B130B2
:100FDD007502C281305A0EE525600A207502D28154
:100FED00307502D2B1207503759F01307503759F61
:100FFD0003753D01D2AF229001D1C2B1C287C2812A
:10100D00C282C286C28022C3E54F9535E550953622
:10101D005001227890E6FFC3EF94055018C3EF946A
:10102D0004501BC3EF9403501EC3EF94025021C311
:10103D00EF94015024C3E54F943CF802106FC3E5C3
:10104D004F9428F802106FC3E54F941AF802106FF1
:10105D00C3E54F9412F802106FC3E54F940AF802DE
:0F106D00106FE5509400F9884F895022305803D6
:10107C00021079227880760778817607788276015B
:10108C00788476037883760178867609788F760172
:10109C00789076057895760278927603789B760D23
:1010AC007893760678877601789C76027888760134
:1010BC007889760178857600788C7601788D760043
:1010CC00788E76B478967625789776D078987678E8
:1010DC00789976C8789A7604789D7600227893E68B
:1010EC00FF756409756501C3BF02097564057565F3
:1010FC000102112EC3BF0309756405756502021147
:10110C002EC3BF040975640575650302112EC3BF98
:10111C000506756409756507C3BF06067564007519
:10112C0065007887E6FFC26CC3BF0302D26CC26B4A
:10113C00C3BF0402D26BC26A7418552D6002D26A06
:10114C00C26E6002D26ED26F6002C26FC2757888B6
:10115C00E630E102D275C2767889E630E102D276C9
:10116C00C3EF94026008758E01D26D02117F758EEB
:10117C0000C26D227880E61490008093789EF678F9
:10118C0081E61490008093789FF6110422789BE6F8
:10119C001490008D9378A0F61104227886E61490B2
:1011AC00009A9378A1F6110422789CE6149000A77B
:1011BC009378A2F6789CE6149000AC9378A3F61181
:1011CC000422227896E6FA7897E6FB3077047A00C8
:1011DC007BFFC3EB9AFCC3948250027C82756C003B
:1011EC00056CEC856CF0A4C3E5F0948040F222C24F
:1011FC00D353D9BF7581C043FF8012075775EF02D7
:10120C0043B203E5B324044002F5B375803875A4EA
:10121C00C775F1FF75D4DF7590FF75A50075F200E9
:10122C0075D50075A0FF75A60075F30075D6007511
:10123C00B0E475A71B75F4FF75E2411104E4F8F6F0
:10124C00D8FD118012178411E93180319931A73101
:10125C00B531CE31CF7898866D110475885075896B
:10126C000275C82475910475D84012076B12077A61
:10127C0012076312078112076312078812076312A1
:10128C001CE512076B12076B12076775A82275B85D
:10129C000275E69075F610759B80759D0375D10EE1
:1012AC0075BC5875BB0675BA1F75E880120757D206
:1012BC00AF120A3343DA01C2D8C26912076B753018
:1012CC0001D2597A05E55770027A0512075BE55889
:1012DC00C3940240EEE52E541F855A59F55AB55960
:1012EC00E2DAE2C25953DACF20760343DA203076C1
:1012FC000343DA10C2D8C26912076712075B78027F
:10130C00741F552E70027800C3E5589840EDC2AF9B
:10131C0012077A12077A12077AD2AF12076B754747
:10132C000012075B788CE6C3940150030213F6E5B8
:10133C0030C3940150030213F6741F552E6035C34D
:10134C00E55894FF50030213F6C2AF12078FD2AFC9
:10135C00120767C3E558940150EFC2AF12077A1217
:10136C00075F12077AD2AF120767C3E55894FF40A4
:10137C00E9021D6A7F05D27731CF120767C2AFC26F
:10138C007731CFC3E558947FD2AF4068C2AF120714
:10139C008FD2AFDFE1C3E55894057897F612076B4F
:1013AC00121833121CED7F0AD27731CF120767C2A5
:1013BC00AFC27731CFC3E558947FD2AF50E8C2AFFC
:1013CC0012077A12075F12077AD2AFDFDBE55824D7
:1013DC00057896F612076B121833121D1C1207674C
:1013EC00C3E55894FF40F6021D6AC3E55895474083
:1013FC0003855847120767C3E55894014002612DD5
:10140C00C2AF12078F12078F12078FD2AF12076B62
:10141C00753000E4F531F5320531E531F4703605FF
:10142C0032789AE67828146012785014600D78A0FF
:10143C0014600878F0146003753200C3E5329840EC
:10144C001415327899866DC2AF12078FD2AF789887
:10145C00866D12076712075BE5287008741F552EFE
:0E146C00700241CDC3E558940640AD120767EB
:10147A00E52870030212CD1104E4F522F523F524C0
:10148A00F525755CFF7885865FF53FF540F541F5F2
:10149A0042F543F56AF548F52BF52CF55B120BB4CA
:1014AA00756A0875BB1E120757120AC8E5E820ECD0
:1014BA00FBA8BDA9BEE97001F8886B120ACC756A4F
:1014CA000875BB1E7895E630E0030215137887E6A7
:1014DA00FE760211E97887EEF6D261C2AF120B846A
:1014EA0085225C85225DD2AFC261752500756200D6
:1014FA00756301D260D263753800120F6F120FAA9A
:10150A00120C30120BB402163C7887E6FE7603788A
:10151A0093E6FD760511E97887EEF67893EDF6D233
:10152A0060D261D26E120F6F120FAA120B841207C9
:10153A0057120E77120757120757120EA912075B96
:10154A00120EF312075B12075B120F2E12075F12BD
:10155A000F6F12075B120757C261D262120AC812D2
:10156A000ACC120B84756A0875BB1E120FAA120CDC
:10157A0029120CA411141179120E77120C29120CCB
:10158A00A411141179120EA9120C29120CA4111407
:10159A001179120EF3120C29120CA41114117912DA
:1015AA000F2E120C29120CA411141179120F6F129A
:1015BA000C29120CA41114C3E54F9535E550953644
:1015CA00400C1179C3E558940150910217561179CC
:1015DA00C2627887E6FE760211E97887EEF68522FE
:1015EA005C855E5D855E25756200756301D26375F3
:1015FA003800C2AF207502C282307502C2802075DF
:10160A0002C280307502C282742DD5E0FDD2AF12BB
:10161A000FAA120C30120C8B120CA4120D28756A28
:10162A000075BB0602163C11E9120FAA756A00750D
:10163A00BB06120D4A120DD4120DFC120879120EB5
:10164A0010120E77120C30120C8B120CA4120D28E9
:10165A00120D41120DD4120DFC1208D7120E1012DF
:10166A000EA9120C30120C8B120CA4120D28120D9A
:10167A004A120DD4120DFC120910120E10120EF39A
:10168A00120C30120C8B120CA4120D28120D4112DE
:10169A000DD4120DFC12096D120E10120F2E120C1F
:1016AA0030120C8B120CA4120D28120D4A120DD4F2
:1016BA00120DFC1209D1120E10120F6F120C3012F9
:1016CA000C8B120CA4120D28120D41120AC8120D0D
:1016DA00D4120DFC120ACC120E10120FAA120C30E0
:1016EA00120C8B120CA4120D2830632A855E5C85BD
:1016FA005E5D756200756301C3E5389464400AC291
:10170A0063D264753714021720C3E5589401400365
:10171A0002163C021756306419E537147005C26484
:10172A00021631F537C3E5589401400302163C020C
:10173A001756C3E55B94FA5013741F552E7004E5CF
:10174A00286009C3E53C94F05002C13C1104788733
:10175A00E6FE760211E97887EEF6E4F522F523F53E
:10176A0024F525F55FC2601207571104741F552E20
:10177A007006E528700241CD811F901A0D7820125B
:10178A001C00E520B4550CA3121C00E520B4AA03E2
:10179A000217A51180121833021832901A037880A2
:1017AA00121C00A308121C00A308121C00901A069F
:1017BA007883121C00A308121C00A308A308121C99
:1017CA0000A308121C00A308121C00A308121C0084
:1017DA00A308A308A308121C00A308A308121C004C
:1017EA00A308121C00A308121C00A308A308121CB9
:1017FA0000A308121C00A308A308121C00A30812C5
:10180A001C00A308121C00A308121C00A308121C27
:10181A0000A308121C00A308121C00A308121C0033
:10182A00A308121C00901A2122C2AF121C3F121CDC
:10183A0019901A00740A121C05A37404121C05A339
:10184A007410121C05901A037880121C04A3081243
:10185A001C04A308121C04901A067883121C04A301
:0D186A0008121C04A308A308121C04A30804
:10187700121C04A308121C04A308121C04A308A327
:1018870008A308121C04A308A308121C04A3081227
:101897001C04A308121C04A308A308121C04A30811
:1018A700121C04A308A308121C04A308121C04A3F7
:1018B70008121C04A308121C04A308121C04A30882
:1018C700121C04A308121C04A308121C04A3081268
:0C18D7001C04121C52121C30901A21221A
:101A00000A04100909040103FF0901010155AA0193
:101A1000FFFF0105FF0306FF0225D02850040D0239
:021A200000FFC5
:101A4000235475726E696779343041232020202039
:101A500023424C48454C4923463331302320202033
:101A60002020202020202020202020202020202076
:101C0000E493F622E6438F01538FFD75EF0275B71B
:101C1000A575B7F1F0538FFE22438F02438F0175F4
:101C2000EF0275B7A575B7F1901A0DF0538FFC222E
:101C3000901A0D74559105901A0E74AA9105227A86
:101C40003079D07820901A409100E520F709A3DA86
:101C5000F7227A3079D0901A40E7910509A3DAF992
:101C600022AB6EA86FBB01057980021CE2BB0205A6
:101C70007981021CE2BB03057982021CE2BB0405E8
:101C80007984021CE2BB05057983021CE2BB0605D0
:101C90007995021CE2BB07057986021CE2BB0805A8
:101CA000798F021CE2BB09057990021CE2BB0A0590
:101CB0007992021CE2BB0B05799B021CE2BB0C056E
:101CC0007993021CE2BB0D057987021CE2BB0E056D
:101CD000799C021CE2BB0F057988021CE27989021B
:101CE0001CE2E8F7227C0512076BDCFB22C2AF1274
:101CF000077A12078112078812078F12075F1207EF
:101D00007A12078112078812078F12075F12077A6B
:101D100012078112078812078FD2AF22C2AF1207B3
:101D20008F12078812078112077A12075F12078F36
:101D300012078812078112077A12075F12078F12A3
:101D4000078812078112077AD2AF22AE6EAF6FC238
:101D5000AF12077A12077A12077A12075FDEF212C1
:101D6000078F12075FDFF8D2AF2291ED91E591E581
:101D7000756E01756F01757000B14B7C05AD581221
:101D8000076BC3ED955870F5C3E55894014009C33E
:101D9000E55894FF4032A1A6916112183391EDC22B
:101DA000AF75EF1291E5DCD50570C3E57094035073
:101DB0000280C691E5056FE56E149000B193F808B6
:101DC000C3E56F98500280AE91E591E5056EC3E5DD
:101DD0006E94115002809C121080121833C2AF759D
:041DE000EF1291E588
:00000001FF
